:0200000077285F
:08000800FF0003088301FE0064
:100010000A08FD0000308A00E12803178D0003174D
:1000200083168C130C1483120C088D0A7328031783
:100030008C0083168C130C1555308D00AA308D0062
:100040008C148C1821280C1183128D0A7328003807
:1000500003193F28A8002008840021188317A10154
:10006000A001A81B3B280008A000A81C3F28840A68
:100070000008A1003F2840200005031DA00A7328A6
:1000800000308A002808073982070134023404341A
:1000900008341034203440348034013EA7000A3044
:1000A000A200A3015720A70B522824080800A5018D
:1000B000A4011030A600210DA40DA50D2208A40254
:1000C0002308031C230FA50203186D282208A40788
:1000D00023080318230FA5070310A00DA10DA60BDD
:1000E0005B282008732883138312031308008316E8
:1000F000811307309C009F008601F0308700073095
:1001000088008312FF30860087018801F930AA0039
:10011000A430AB00B030AC009930AD009230AE00EE
:100120008230AF00F830B0008030B1009030B200C3
:10013000C030B300BF30B4007F30B50088308316C4
:100140008100EF30831281008B168B1700308A01FB
:100150000D20CD0001308A010D20CE00D201D10149
:100160000C30D0001C30CF005208C1005108C00034
:100170005008BF004F08BE004C108A110A12C02858
:1001800088128A150A120F22C3014D08C2008A1173
:100190000A12071ECE288A110A1232298A110A125F
:1001A000871BD5288A110A12612E8A110A12081C8F
:1001B000DC288A150A124D218A110A127E278A012B
:1001C000C7288A110A124C18E8288A110A1227290E
:1001D0000130BE020301031C0130BF020301031CF6
:1001E0000130C0020301031C0130C1028A110A124E
:1001F000C11B05293E083F04400441048A110A122C
:10020000031905298A110A122729410840043F04CD
:100210003E048A110A12031D1B294F08BE0750080D
:100220000318500FBF0751080318510FC007520899
:100230000318520FC107C3038A110A12C31F2129D1
:10024000C2038A110A12C31F27293B30C3000B11B6
:100250007D088A007E088300FF0E7F0E0900630080
:100260008A012F298A110A124C1C38298A01C728B1
:100270004C108A110A127E27881508178A110A1253
:10028000871E45298A110A12612E8A110A12871BBC
:100290004C298A110A12612E8A110A12071B52294F
:1002A0008A0132294D03C2003B30C3004C1442087E
:1002B000A000A10100308A014D20C4004208A00026
:1002C000A10101308A014D20C5004308A000A10111
:1002D00000308A014D20C6004308A000A101013072
:1002E0008A014D20C700013043020130031D003058
:1002F000A9000130C408031D0030A9058A110A12A3
:10030000031985298A110A125C2B4408A200093CB2
:100310008A110A12031CC5290310220DA2078A1193
:100320000A12A321A000A20A8A110A12A321A10085
:10033000A20A8A110A12A3218A0127202008C800D4
:100340008A110A12C52901308A0022088207333433
:10035000003401342A34003401342B3400340134A5
:100360002C34003401342D34003401342E34003464
:1003700001342F340034013430340034013431344A
:10038000003401343234003401344508A200093C01
:100390008A110A12031C1F2A0310220DA2078A11B8
:1003A0000A12E321A000A20A8A110A12E321A10085
:1003B000A20A8A110A12E3218A0127202008C90013
:0E03C0008A110A121F2A02308A002208002A1F
:1004000082073334003401342A34003401342B346D
:10041000003401342C34003401342D3400340134E0
:100420002E34003401342F3400340134303400349D
:10043000013431340034013432340034013446089C
:10044000A200093C8A110A12031C5F2A0310220D24
:10045000A2078A110A123D22A000A20A8A110A12DA
:100460003D22A100A20A8A110A123D228A012720F8
:100470002008CA008A110A125F2A02308A00220864
:1004800082073334003401342A34003401342B34ED
:10049000003401342C34003401342D340034013460
:1004A0002E34003401342F3400340134303400341D
:1004B000013431340034013432340034013447081B
:1004C000A200093C8A110A12031C9F2A0310220D64
:1004D000A2078A110A127D22A000A20A8A110A121A
:1004E0007D22A100A20A8A110A127D228A012720F8
:1004F0002008CB008A110A129F2A02308A002208A3
:1005000082073334003401342A34003401342B346C
:10051000003401342C34003401342D3400340134DF
:100520002E34003401342F3400340134303400349C
:1005300001343134003401343234003401340130B8
:10054000870049088600B901B801B701B6018A11D0
:100550000A12B91BB82A3708380439048A110A125A
:10056000031DCA2A0B3036028A110A120318CA2A3E
:100570000130B607030103180130B7070301031860
:100580000130B807030103180130B9078A110A12B4
:10059000031CA72A02308700803048078600B90173
:1005A000B801B701B6018A110A12B91BE42A37084B
:1005B000380439048A110A12031DF62A0B30360258
:1005C0008A110A120318F62A0130B607030103182C
:1005D0000130B707030103180130B80703010318FE
:1005E0000130B9078A110A12031CD32A0830870088
:1005F0004A088600B901B801B701B6018A110A128A
:10060000B91B0F2B3708380439048A110A12031D4D
:10061000212B0B3036028A110A120318212B0130CC
:10062000B607030103180130B707030103180130AF
:10063000B807030103180130B9078A110A12031C15
:10064000FE2A043087004B088600B901B801B701C3
:10065000B6018A110A12B91B3A2B3708380439043B
:100660008A110A12031D4C2B0B3036028A110A1212
:1006700003184C2B0130B607030103180130B707EC
:10068000030103180130B807030103180130B9074B
:100690008A110A12031C292B8A110A12871E532B56
:1006A0008A110A12612E8A110A12871B5A2B8A118B
:1006B0000A12612E8A0157294C1088110816081356
:1006C00088178A110A12871E682B8A110A12612E56
:1006D0008A110A12871B6F2B8A110A12612ECE080B
:1006E0008A110A12031D772B8A150A12F8294E0364
:1006F000C2003B30C3004C144208A000A1010030EE
:100700008A014D20C4004208A000A10101308A01E5
:100710004D20C5004308A000A10100308A014D20F2
:10072000C6004308A000A10101308A014D20C70086
:100730000130C408031D0030A9000130430201301C
:10074000031D0030A9058A110A120319AA2B8A1564
:100750000A12F8294408A200093C8A110A12031C53
:10076000EA2B0310220DA2078A110A12C823A00047
:10077000A20A8A110A12C823A100A20A8A110A1227
:10078000C8238A0127202008C8008A110A12EA2BF0
:1007900003308A00220882073334003401342A34BB
:1007A000003401342B34003401342C34003401344F
:1007B0002D34003401342E34003401342F3400340D
:1007C00001343034003401343134003401343234F3
:1007D000003401344508A200093C8A110A12031CA6
:1007E0002A2C0310220DA2078A110A120824A00045
:1007F000A20A8A110A120824A100A20A8A110A1266
:1008000008248A0127202008C9008A110A122A2CEC
:1008100004308A00220882073334003401342A3439
:10082000003401342B34003401342C3400340134CE
:100830002D34003401342E34003401342F3400348C
:100840000134303400340134313400340134323472
:10085000003401344608A200093C8A110A12031C24
:100860006A2C0310220DA2078A110A124824A00044
:10087000A20A8A110A124824A100A20A8A110A12A5
:1008800048248A0127202008CA008A110A126A2CEB
:1008900004308A00220882073334003401342A34B9
:1008A000003401342B34003401342C34003401344E
:1008B0002D34003401342E34003401342F3400340C
:1008C00001343034003401343134003401343234F2
:1008D000003401344708A200093C8A110A12031CA3
:1008E000AA2C0310220DA2078A110A128824A00044
:1008F000A20A8A110A128824A100A20A8A110A12E5
:1009000088248A0127202008CB008A110A12AA2CE9
:1009100004308A00220882073334003401342A3438
:10092000003401342B34003401342C3400340134CD
:100930002D34003401342E34003401342F3400348B
:100940000134303400340134313400340134323471
:1009500000340134BD01BC01BB01BA018A110A1285
:10096000BD1BBF2C3B083C043D048A110A12031D29
:100970007E2D33303A028A110A1203187E2D01307F
:10098000870049088600B901B801B701B6018A118C
:100990000A12B91BD82C3708380439048A110A12F4
:1009A000031DEA2C0B3036028A110A120318EA2CB6
:1009B0000130B607030103180130B707030103181C
:1009C0000130B807030103180130B9078A110A1270
:1009D000031CC72C02308700803048078600B9010D
:1009E000B801B701B6018A110A12B91B042D3708E4
:1009F000380439048A110A12031D162D0B303602F1
:100A00008A110A120318162D0130B60703010318C4
:100A10000130B707030103180130B80703010318B9
:100A20000130B9078A110A12031CF32C0830870021
:100A30004A088600B901B801B701B6018A110A1245
:100A4000B91B2F2D3708380439048A110A12031DE7
:100A5000412D0B3036028A110A120318412D013044
:100A6000B607030103180130B7070301031801306B
:100A7000B807030103180130B9078A110A12031CD1
:100A80001E2D043087004B088600B901B801B7015C
:100A9000B6018A110A12B91B5A2D370838043904D5
:100AA0008A110A12031D6C2D0B3036028A110A12AC
:100AB00003186C2D0130B607030103180130B70786
:100AC000030103180130B807030103180130B90707
:100AD0008A110A12031C492D0130BA0703010318B9
:100AE0000130BB07030103180130BC0703010318E1
:100AF0000130BD078A110A12031CAE2CBD01BC01D6
:100B0000BB01BA018A110A12BD1B932D3B083C049C
:100B10003D048A110A12031D512E65303A028A11D2
:100B20000A120318512E0130870049088600B901C6
:100B3000B801B701B6018A110A12B91BAC2D3708EA
:100B4000380439048A110A12031DBE2D0B303602F7
:100B50008A110A120318BE2D0130B60703010318CB
:100B60000130B707030103180130B8070301031868
:100B70000130B9078A110A12031C9B2D023087002D
:100B800048088600B901B801B701B6018A110A12F6
:100B9000B91BD72D3708380439048A110A12031DEE
:100BA000E92D0B3036028A110A120318E92D0130A3
:100BB000B607030103180130B7070301031801301A
:100BC000B807030103180130B9078A110A12031C80
:100BD000C62D083087004A088600B901B801B70160
:100BE000B6018A110A12B91B022E370838043904DB
:100BF0008A110A12031D142E0B3036028A110A12B2
:100C00000318142E0130B607030103180130B7078B
:100C1000030103180130B807030103180130B907B5
:100C20008A110A12031CF12D043087004B0886003C
:100C3000B901B801B701B6018A110A12B91B2D2EEC
:100C40003708380439048A110A12031D3F2E0B306D
:100C500036028A110A1203183F2E0130B60703012B
:100C600003180130B707030103180130B807030167
:100C700003180130B9078A110A12031C1C2E013017
:100C8000BA07030103180130BB0703010318013041
:100C9000BC07030103180130BD078A110A12031CA7
:100CA000822D8A110A12871E582E8A110A12612E6D
:100CB0008A110A12871B5F2E8A110A12612E8A017D
:100CC0007C2B88110812081388134C10FF30C800C1
:100CD0008630C900AF30CA002F30CB00BD01BC0147
:100CE000BB01BA018A110A12BD1B832E3B083C04CA
:100CF0003D048A110A12031D422F65303A028A11FF
:100D00000A120318422F0130870048088600B901F3
:100D1000B801B701B6018A110A12B91B9C2E370817
:100D2000380439048A110A12031DAE2E0B30360224
:100D30008A110A120318AE2E0130B60703010318F8
:100D40000130B707030103180130B8070301031886
:100D50000130B9078A110A12031C8B2E023087005A
:100D600049088600B901B801B701B6018A110A1213
:100D7000B91BC72E3708380439048A110A12031D1B
:100D8000D92E0B3036028A110A120318D92E0130DF
:100D9000B607030103180130B70703010318013038
:100DA000B807030103180130B9078A110A12031C9E
:100DB000B62E083087004B088600B901B801B7018C
:100DC000B6018A110A12B91BF22E37083804390409
:100DD0008A110A12031D042F0B3036028A110A12DF
:100DE0000318042F0130B607030103180130B707B9
:100DF000030103180130B807030103180130B907D4
:100E00008A110A12031CE12E043087004A0886006A
:100E1000B901B801B701B6018A110A12B91B1D2F19
:100E20003708380439048A110A12031D2F2F0B309A
:100E300036028A110A1203182F2F0130B607030158
:100E400003180130B707030103180130B807030185
:100E500003180130B9078A110A12031C0C2F8816D7
:100E60000130BA07030103180130BB07030103185F
:100E70000130BC07030103180130BD078A110A12B3
:100E8000031C722EBD01BC01BB01BA018A110A12FA
:100E9000BD1B602F3C083D048A110A12031D762FEA
:100EA0003B08273C8A110A12031C762F8A110A126A
:100EB000031D602F3A08103C8A110A12031C762F7A
:100EC0008701FF30860088120130BA07030103183A
:100ED0000130BB07030103180130BC0703010318ED
:100EE0000130BD078A110A12031C462F8A110A120B
:100EF000871E7C2F8A01C0288A01612E4208A0002B
:100F0000A10100308A014D20C4004208A000A101C7
:100F100001308A014D20C5004308A000A101003026
:100F20008A014D20C6004308A000A10101308A01BA
:100F30004D20C7004408A200093C8A110A12031C74
:100F4000DA2F0310220DA2078A110A12B827A00077
:100F5000A20A8A110A12B827A100A20A8A110A124B
:100F6000B8278A0127202008C8008A110A12DA2F20
:100F700007308A00220882073334003401342A34CF
:100F8000003401342B34003401342C340034013467
:100F90002D34003401342E34003401342F34003425
:100FA000013430340034013431340034013432340B
:100FB000003401344508A200093C8A150A12031CBA
:100FC0001F280310220DA2078A110A12F827A00079
:100FD000A20A8A110A12F827A100A20A8A110A128B
:100FE000F8278A0127202008C9008A150A121F281D
:080FF00008308A0022080028E5
:1010000082073334003401342A34003401342B3461
:10101000003401342C34003401342D3400340134D4
:101020002E34003401342F34003401343034003491
:101030000134313400340134323400340134460890
:10104000A200093C8A150A12031C5F280310220D16
:10105000A2078A150A123D20A000A20A8A150A12C8
:101060003D20A100A20A8A150A123D208A012720EC
:101070002008CA008A150A125F2808308A00220850
:1010800082073334003401342A34003401342B34E1
:10109000003401342C34003401342D340034013454
:1010A0002E34003401342F34003401343034003411
:1010B000013431340034013432340034013447080F
:1010C000A200093C8A150A12031C9F280310220D56
:1010D000A2078A150A127D20A000A20A8A150A1208
:1010E0007D20A100A20A8A150A127D208A012720EC
:1010F0002008CB008A150A129F2808308A0022088F
:1011000082073334003401342A34003401342B3460
:10111000003401342C34003401342D3400340134D3
:101120002E34003401342F34003401343034003490
:1011300001343134003401343234003401340130AC
:10114000870049088600B901B801B701B6018A15C0
:101150000A12B91BB8283708380439048A150A124C
:10116000031DCA280B3036028A150A120318CA2832
:101170000130B607030103180130B7070301031854
:101180000130B807030103180130B9078A150A12A4
:10119000031CA72802308700803048078600B90169
:1011A000B801B701B6018A150A12B91BE42837083D
:1011B000380439048A150A12031DF6280B3036024A
:1011C0008A150A120318F6280130B607030103181E
:1011D0000130B707030103180130B80703010318F2
:1011E0000130B9078A150A12031CD328083087007A
:1011F0004A088600B901B801B701B6018A150A127A
:10120000B91B0F293708380439048A150A12031D3F
:1012100021290B3036028A150A12031821290130C0
:10122000B607030103180130B707030103180130A3
:10123000B807030103180130B9078A150A12031C05
:10124000FE28043087004B088600B901B801B701B9
:10125000B6018A150A12B91B3A293708380439042D
:101260008A150A12031D4C290B3036028A150A1200
:1012700003184C290130B607030103180130B707E2
:10128000030103180130B807030103180130B9073F
:101290008A150A12031C292908008A150A124C1CF7
:1012A00052290800C3014D08C2008A150A12F32210
:1012B0008A017E278A150A12881C5F29C20A8A15AC
:1012C0000A12081D6429C203BD01BC01BB01BA0199
:1012D0008A150A12BD1B79293B083C043D048A1576
:1012E0000A12031D8D2965303A028A150A12031865
:1012F0008D298A017E270130BA07030103180130C6
:10130000BB07030103180130BC07030103180130B8
:10131000BD078A150A12031C68298A150A120818C3
:1013200094298A150A1258294208CD004E08C20095
:101330008A150A12D8238A017E278A150A12881C68
:10134000A229C20A643042028A150A12031DA92981
:10135000C2038A150A12081DAE29C2038A150A1291
:10136000C21FB329C20ABD01BC01BB01BA018A1563
:101370000A12BD1BC8293B083C043D048A150A1209
:10138000031DDC2965303A028A150A120318DC298C
:101390008A017E270130BA07030103180130BB0719
:1013A000030103180130BC07030103180130BD0716
:1013B0008A150A12031CB7298A150A120818E3298C
:1013C0008A150A129B294208CE008A150A120F229A
:1013D0004D08C20003178D0103134D088A01172021
:1013E000013003178D0003134E088A0117200800EF
:1013F00088110812881688134C108A150A12871E45
:10140000032A8A01C0288A150A12871B092A8A0121
:10141000612E8A150A12BD248A150A12F829C230D3
:10142000C800A330C900CA002130CB00BD01BC01F7
:10143000BB01BA018A150A12BD1B342A3C083D04BF
:101440008A150A12031DF22A3B08033C8A150A1268
:10145000031CF22A8A150A12031D342A3A08E83CB2
:101460008A150A12031CF22A0130870048088600F8
:10147000B901B801B701B6018A150A12B91B4D2A84
:101480003708380439048A150A12031D5F2A0B3005
:1014900036028A150A1203185F2A0130B6070301C3
:1014A00003180130B707030103180130B80703011F
:1014B00003180130B9078A150A12031C3C2A0230AE
:1014C000870049088600B901B801B701B6018A153D
:1014D0000A12B91B782A3708380439048A150A1207
:1014E000031D8A2A0B3036028A150A1203188A2A2B
:1014F0000130B607030103180130B70703010318D1
:101500000130B807030103180130B9078A150A1220
:10151000031C672A083087004B088600B901B80110
:10152000B701B6018A150A12B91BA32A3708380475
:1015300039048A150A12031DB52A0B3036028A15A2
:101540000A120318B52A0130B60703010318013047
:10155000B707030103180130B8070301031801306E
:10156000B9078A150A12031C922A043087004A0818
:101570008600B901B801B701B6018A150A12B91B74
:10158000CE2A3708380439048A150A12031DE02AC6
:101590000B3036028A150A120318E02A0130B6070A
:1015A000030103180130B707030103180130B8071E
:1015B000030103180130B9078A150A12031CBD2A5A
:1015C0000130BA07030103180130BB0703010318F8
:1015D0000130BC07030103180130BD078A150A1248
:1015E000031C1A2A08009230C8008630C9008730D0
:1015F000CA002A08CB00BD01BC01BB01BA018A1593
:101600000A12BD1B192B3C083D048A150A12031D42
:10161000D72B3B08033C8A150A12031CD72B8A15CB
:101620000A12031D192B3A08E83C8A150A12031CFA
:10163000D72B0130870048088600B901B801B701EF
:10164000B6018A150A12B91B322B3708380439043F
:101650008A150A12031D442B0B3036028A150A1212
:101660000318442B0130B607030103180130B707F4
:10167000030103180130B807030103180130B9074B
:101680008A150A12031C212B0230870049088600A4
:10169000B901B801B701B6018A150A12B91B5D2B51
:1016A0003708380439048A150A12031D6F2B0B30D2
:1016B00036028A150A1203186F2B0130B607030190
:1016C00003180130B707030103180130B8070301FD
:1016D00003180130B9078A150A12031C4C2B083075
:1016E00087004B088600B901B801B701B6018A1519
:1016F0000A12B91B882B3708380439048A150A12D4
:10170000031D9A2B0B3036028A150A1203189A2BE6
:101710000130B607030103180130B70703010318AE
:101720000130B807030103180130B9078A150A12FE
:10173000031C772B043087004A088600B901B801E2
:10174000B701B6018A150A12B91BB32B3708380442
:1017500039048A150A12031DC52B0B3036028A156F
:101760000A120318C52B0130B60703010318013014
:10177000B707030103180130B8070301031801304C
:10178000B9078A150A12031CA22B0130BA070301FC
:1017900003180130BB07030103180130BC07030124
:1017A00003180130BD078A150A12031CFF2A08001E
:1017B0009230C8008630C9008730CA002B08CB00A1
:1017C000BD01BC01BB01BA018A150A12BD1BFE2B6B
:1017D0003C083D048A150A12031DBC2C3B08033C3F
:1017E0008A150A12031CBC2C8A150A12031DFE2B33
:1017F0003A08E83C8A150A12031CBC2C0130870009
:1018000048088600B901B801B701B6018A150A1265
:10181000B91B172C3708380439048A150A12031D1E
:10182000292C0B3036028A150A120318292C013094
:10183000B607030103180130B7070301031801308D
:10184000B807030103180130B9078A150A12031CEF
:10185000062C0230870049088600B901B801B7019B
:10186000B6018A150A12B91B422C3708380439040C
:101870008A150A12031D542C0B3036028A150A12DF
:101880000318542C0130B607030103180130B707C1
:10189000030103180130B807030103180130B90729
:1018A0008A150A12031C312C083087004B08860069
:1018B000B901B801B701B6018A150A12B91B6D2C1E
:1018C0003708380439048A150A12031D7F2C0B309F
:1018D00036028A150A1203187F2C0130B60703015D
:1018E00003180130B707030103180130B8070301DB
:1018F00003180130B9078A150A12031C5C2C043046
:1019000087004A088600B901B801B701B6018A15F7
:101910000A12B91B982C3708380439048A150A12A0
:10192000031DAA2C0B3036028A150A120318AA2CA2
:101930000130B607030103180130B707030103188C
:101940000130B807030103180130B9078A150A12DC
:10195000031C872C0130BA07030103180130BB07B1
:10196000030103180130BC07030103180130BD0750
:101970008A150A12031CE42B0800FF30C8008630C9
:10198000C900AB30CA002130CB00013087004808C5
:101990008600B901B801B701B6018A150A12B91B50
:1019A000DE2C3708380439048A150A12031DF02C7E
:1019B0000B3036028A150A120318F02C0130B607D4
:1019C000030103180130B707030103180130B807FA
:1019D000030103180130B9078A150A12031CCD2C24
:1019E0000230870049088600B901B801B701B60185
:1019F0008A150A12B91B092D3708380439048A15CB
:101A00000A12031D1B2D0B3036028A150A12031809
:101A10001B2D0130B607030103180130B70703017E
:101A200003180130B807030103180130B9078A15FC
:101A30000A12031CF82C083087004B088600B901F5
:101A4000B801B701B6018A150A12B91B342D37083F
:101A5000380439048A150A12031D462D0B3036024C
:101A60008A150A120318462D0130B6070301031820
:101A70000130B707030103180130B8070301031849
:101A80000130B9078A150A12031C232D0430870080
:101A90004A088600B901B801B701B6018A150A12D1
:101AA000B91B5F2D3708380439048A150A12031D43
:101AB000712D0B3036028A150A120318712D013070
:101AC000B607030103180130B707030103180130FB
:101AD000B807030103180130B9078A150A12031C5D
:0A1AE0004E2D08008A150A12722D1F
:02400E00323F3F
:00000001FF
